:1000000000308A006C290000831685118312851147
:10001000A6308C008C0B0A28000083168515A630AC
:1000200083128C008C0B1228000083168515831216
:100030000034A4012408073C031C3B2883168511C7
:1000400083128511000000000314A30C03182A2852
:1000500085112B28851583168511133083128C008A
:100060008C0B30280000000083168515000000006E
:100070008312A40A1A280034A3012308073C031C96
:1000800060288316851183128511000000008316F5
:100090008515023083128C008C0B4C2800008316CF
:1000A0008515831285195628031057280314A40CAC
:1000B00027308C008C0B5A2800000000A30A3D2832
:1000C00024088D000034240826068039A800A41FC7
:1000D0006E28A309A409A30A0319A40AA61F752858
:1000E000A509A609A50A0319A60A8D018E018C018E
:1000F0008F012608031D7F28250803199928103031
:10010000A7000310A30DA40D8C0D8F0D26080F0260
:10011000031D8C2825080C02031C952825088C0239
:10012000031C8F0326088F0203148D0D8E0DA70B61
:1001300081280000A81FA1288D098E098D0A0319A6
:100140008E0AE8288E308C0024088D0023088E004B
:100150008F018D08031DB6280E088D008E01083012
:100160008C028D08031DB6288C01BE2803108D1B40
:10017000BD288E0D8D0D8C03B6288D130000EC2844
:100180009A010420CC30A30019204430A300192088
:100190009A08031DCF283C200D089A00C828042087
:1001A000CC30A3001920BE30A30019203C200D083C
:1001B0009B003C200D089C001C089E001B089D0015
:1001C0001E08A4001D08A300A6011030A500632886
:1001D0000D08A401A300A2280F08A2000E08A10088
:1001E0000D08A0000C089F001F088C0020088D003F
:1001F00021088E0022088F0076298E308C001A0884
:100200008C021B088E001C088D008E178C080319A9
:10021000142903108E08031D10298D0803191429B1
:100220008E0C8D0C8C0B09299B1F1B298D098E09A7
:100230008D0A03198E0A00007F291B088D011A02FE
:10024000031825291A088C0031298C0108309C00DC
:100250009A0D8C0D1B080C0203188C008D0D9C0B45
:1002600028298E298C018D011A0803101B188C0770
:100270008C0C8D0C9B188C078C0C8D0C1B198C070F
:100280008C0C8D0C9B198C078C0C8D0C1B1A8C07FD
:100290008C0C8D0C9B1A8C078C0C8D0C1B1B8C07EB
:1002A0008C0C8D0C9B1B8C078C0C8D0C95291A309B
:1002B0008400000803196B2901308D008C018C0B20
:1002C0005F298D0B5E294A308C008C0B652900005C
:1002D0000000800B5C29102A84011F3083058316DF
:1002E0000108C739083881008312C0280F089D0013
:1002F0000E089C000D089B000C089A00FD280D08B4
:1003000094001408093C031C8929140895009601DF
:10031000982914089A000A309B001D290D089600A0
:1003200016089A000A309B0032290D081402950025
:1003300098011808013C031C122A9808031DAA29D9
:1003400083168510831285108316051183120515F7
:1003500015089700180BB62983160511831205118D
:10036000831685108312851416089700170BBD2974
:1003700083168601F330831286001708023C031DA2
:10038000C629831686014930831286001708033C6C
:10039000031DCF298316860161308312860017085A
:1003A000043C031DD829831686013330831286004E
:1003B0001708053C031DE1298316860125308312A9
:1003C00086001708063C031DEA29831686010530BE
:1003D000831286001708073C031DF3298316860144
:1003E000F130831286001708083C031DFC29831690
:1003F00086010130831286001708093C031D052A77
:10040000831686012130831286009708031D0D2A6A
:10041000831686018130831286000A309A0057299C
:0A042000980A9929831674296300D5
:02400E00F93F78
:00000001FF
